:020000020000FC
:0200000007C037
:02000A00CCC167
:10000E00D6C10FED0DBF00E409B900E007BB0FEF3D
:10001E0008BB0AE501BB09EC02BB539A549A579AE6
:10002E0006E80EBD19D018D03CD140D115D071E0E4
:10003E00A8950FE001BD789452C00F9303E72DD120
:10004E000F910895482C372C262C2A94F1F73A94C8
:10005E00D9F74A94C1F7089502E3602E00E0702E9E
:10006E000FEF802EEFDF0BEE602E05E1702E01E01C
:10007E00802EE8DFA895089500E00DBD0CBDEE279B
:10008E00949A949800E809BF8B989398E5DF9A9418
:10009E00E9F78B9A939A002709BF089501E3FDD0E3
:1000AE00CCDFFFD001E0902EE7DF80D018C001E357
:1000BE00F4D000E3F2D0C1DFF4D00AE0902EDCDF02
:1000CE0075D00DC001E3E9D000E3E7D000E3E5D041
:1000DE00B4DFE7D004E6902ECFDF68D000C0072F44
:1000EE000770003049F00130C9F2023001F30330DD
:1000FE0049F3043061F1F3CF00E3CFD00EE2CDD05F
:10010E0001E3CBD09ADFCDD07F7700E00DBD0CBDE3
:10011E00EE27949A949800E809BF8B98939807D08D
:10012E008B9A939A002709BF02D040D0D8CF02E80D
:10013E00602E0EEF702E0AE0802E84DF01E0602E1E
:10014E0001E0702E05EE802E7DDFA895089574E2F5
:10015E008B989398949A969800E00DBD0CBDEE275F
:10016E00FF2700E809BF74FD18C0AA277F7B2CB5B6
:10017E003DB54E2F5F2FC5D0062F37D0052F35D06A
:10018E00042F33D0032F31D0022F2FD077FDB4D0D0
:10019E0088D09CD0CCDFA895E6CF8B9A939A002777
:1001AE0009BF939A8B9A9498969A99CFAA277F7B98
:1001BE003CB54DB55E2F2FEF00E00DBD0CBD0CB55F
:1001CE00002321F42A959398939AF9CF9AD0062F6B
:1001DE000CD0052F0AD0042F08D0032F06D0022FE3
:1001EE0004D077FD89D05DD008950F9302950F70DE
:1001FE00006339D00F910F70006335D008950F93BF
:10020E00072F0770043009F401E002950A2B023023
:10021E00E1F00530D1F00830C1F00131B1F0043118
:10022E00A1F0073191F0033281F0063271F0023302
:10023E0061F0053351F00A3161F0093251F00833A3
:10024E0041F00A3051F00F9108950CE226D00F9133
:10025E0008950EE222D00F91089500E31ED00EE213
:10026E001CD00F910895A395B72FB770B295BA2BE6
:10027E00B93209F47064B83309F47064003321F0B4
:10028E0070640BD0BCDF089576FF03C006D0B7DFD5
:10029E000895AA3011F000E200C05D9BFECF0CB9AC
:1002AE0008950AE0FADF0DE0F8DF0895EF93FF936B
:1002BE00F2E0EAEC19D0FF91EF91089566666D7445
:1002CE0072303430393136410A0D0000EF93FF930E
:1002DE00F2E0EAEE09D0FF91EF910895436F756E4B
:1002EE0074696E670A0D0000C895002021F0002D7C
:1002FE00D4DF3196F9CF08950F930BE2CEDF0F9135
:10030E0008950F931F937F938F9320D0242F352F13
:10031E00462F572F682F8F917F911F910F91089520
:10032E00042F152F6FEF639500511742E0F75FE929
:10033E00505108511C4FE0F3539504561040E0F70E
:10034E0040EA4051065FE8F3400F0895E9DF772752
:10035E008EEF4D5C43FF435047FF40535D5C53FFB0
:10036E00535057FF50536D5C63FF635067FF6053EC
:10037E00220F331F441F551F661F771F881F4AF316
:10038E00111F18F77D5C73FF735077FF70538D5FED
:10039E0083FF8350DECF0F930FB775FD02C0E39539
:1003AE0001C0319609F470680FBF0F9118950F9325
:1003BE000FB70F930BB10CB10F7D023599F0072FCC
:1003CE0007700395053061F0787F702B706101E046
:1003DE00902E602E702E802E0F910FBF0F911895BC
:1003EE0000E0F2CF072F0770043049F700E00DBD93
:0803FE000CBDEE27FF27F0CF34
:00000001FF
